:10E000000C94417E20202020202020202020202031
:10E0100020202020202020D3FEFD2020D9DA20201F
:10E020002020D9DA202122232425262728292A2B3B
:10E030002C2D2E2F303132333435363738393A3BA8
:10E040003C3D3E3F404142434445464748494A4B98
:10E050004C4D4E4F505152535455565758595A5B88
:10E060005C5D5E5F606162636465666768696A6B78
:10E070006C6D6E6F707172737475767778797A20C3
:10E080002020E92041A042A1E045A3A4A5A64BA7DA
:10E090004D484FA8504354A9AA58E1ABACE2ADAEED
:10E0A000C4AFB0B161B2B3B4E365B6B7B8B9BABB87
:10E0B000BCBD6FBE2020202020202020202020203A
:10E0C0002020202020202020202020202020202050
:10E0D000202020202020202020202020202020FF61
:10E0E000202020207063BF79E478E5C0C1E6C2C378
:10E0F000C4C5C6C7A2B500010203202020202020ED
:10E10000202020200E11101C10110E0000000E11F6
:10E110001C110E000A000E0404040E00000A000C7C
:10E1200004040E00AC1F2001FFFF0000AC1F000123
:10E1300000474B002001436F6E6E65637420776962
:10E1400074682049503A00536561726368207365B2
:10E15000727665722E2E2E0055435320424C20338A
:10E160002E302E302E313120485742205543532E29
:10E170003130382E302E300094A3A6B40B000000AE
:10E18000000003000000006C0000000021063D01BB
:10E1900000003D000001BAFDBA93AA93ABEDB3E0D5
:10E1A00000E012D04FD008C0BA93AA93A801ABEDFB
:10E1B000B3E001E009D005D00E94EB7DA991B991AF
:10E1C0000895E0E5F3E041C0FD0102A702E01FEF82
:10E1D00003A714A700E030E0ECE7F1EEE00FF31F37
:10E1E0001491FD01E00FF31F15A70395003198F37B
:10E1F00003E13A930A936CE477E40895BA93AA93FF
:10E2000033D033E032A7A0E5B3E015963C911996E0
:10E2100033A724A72C911E9735A5322B35A70A5F6B
:10E220001F4F1A930A9350D0C9CF1ED014E012A7E3
:10E2300003A702E002D00C94EB7D10E01A930A933E
:10E240006CE477E4AB01E0E5F3E000811181228129
:10E250003381089509D015E012A703A702E004A7AF
:10E260000FEF05A704E0E6CFEBEDF3E0089521D131
:10E270000FEF0083018302830383048300E005839F
:10E2800002E0068300E00783008701870287048796
:10E290000387058706870895FDD17EDF23C105D159
:10E2A000A0E5B3E0FD0127813085F901E75FFE4F6E
:10E2B00080819181AC0105E014E0F9D09A938A93B2
:10E2C00003D0E4E00C94907E6CE477E4AB010D9114
:10E2D0001D912D913C91AFCF55D00689002300E0D0
:10E2E00011F0068B01E00895392F482F4BD0048997
:10E2F0001589C8010196848B958B0A3020E0104067
:10E3000071F4248B258B02891389012B19F401E008
:10E31000068B05C0028901501040028B138B842F9D
:10E32000932F08959C012ED0002349F00A9561F0A7
:10E330000A95C1F00A9561F00A95C1F007C01BD09B
:10E3400029F400E0C901089516D0D9F301E0FACF0D
:10E350008089918986309040CCF311D00A301140E9
:10E36000A8F7EFCF808991898430F5CF08D00230AB
:10E37000104061F7E6CF03D00331104008950089C3
:10E3800011890895E0E5F3E008951B2F2A2FFADFA5
:10E3900000E0F0D10C9301870287A22FB12F0895DE
:10E3A0001B2F2A2F86D0A781B0850A2F0B2B41F077
:10E3B00000E0A75FBE4F0D930C930783008705878E
:10E3C000ECCF73D0C901F801208126FF03C000E023
:10E3D00010E077CFA0E5B3E0FD012681233019F0EE
:10E3E0000FEF1FEFF6CF202F212B89F3282F232BA0
:10E3F00071F3833020E0920750F327813085232B7F
:10E4000079F72DE331E027833087873021E09207C9
:10E4100038F720E025872387AC01980108E014E055
:10E4200046D00396FD0107811085075F1E4FF80156
:10E4300080839183FD0124818C0106501040DEDE33
:10E4400051D0AC0125E034E0FD01078110852FD0CB
:10E45000BECF2BD0A9012DD021853285622F632B11
:10E4600091F0D9016C9166FD07C06681633021F09F
:10E470001BD00FEF1FEF09C0602F612B19F0642F25
:10E48000652B21F411D000E010E01BCFF901EA5F09
:10E49000FE4F608171814617570750F3CB01AB01E6
:10E4A00006D002D08C01F1CF70CF0C94837E0C94F7
:10E4B0009D7EE0E5F3E00895D7DE05A700E006A71E
:10E4C00007A709E000AB01E001AB25E030E0BD9615
:10E4D0008F0177CF00913905BDDE04D053DF06856B
:10E4E0000860D8CE012B09F0C7D008954BDF058115
:10E4F0000E3F11F401E001C00395058351CF9A93BB
:10E500008A9340E130E006E311EE87D15ADE0E94A3
:10E510003B7BC8010E94D37E402F30E18C0120E07C
:10E520000E94107476D18991999108950E947D7E00
:10E530008EE095E0FC0183A494A402A5A0E5B3E0DD
:10E54000FD0116811A9539F01A9529F01A9539F1BD
:10E550001A9529F18EC0FC01428C538C648C758C09
:10E56000002319F00A9591F084C00AD109F081C006
:10E5700092D009F07EC08ED087D083D0B3DF03E085
:10E58000FD01068301E898DFBADF73C001E0EFD038
:10E5900009F06FC080D009F06CC076D0F0CF0023B6
:10E5A00041F00A9599F0025099F00A9509F45AC081
:10E5B00060C064D0E5D009F05CC06DD009F059C0EE
:10E5C00060D0012B09F455C057D053C057D051C06B
:10E5D00055D0CDD009F044C0FC0103A5002399F427
:10E5E00001E0FD01058300E00483DADE00E01DDECA
:10E5F00079DFFC0105A500FF3CC000E0FD010583BB
:10E6000000E85ADF36C0FD0101851285012B41F576
:10E61000FC0104A545D0FC0113A5FD0104811017E0
:10E62000C1F00685077F06871483408851880DEF67
:10E63000400E0FEF501E96D0A2019C01235D3F4F6C
:10E6400036DFFD01018512850A5F1E4FF801408209
:10E650005182FC0103A5E9DD012B09F0B5CF09C00A
:10E6600039DF07C00BD004E082D019F4FC0103A508
:10E6700017D0EAE00C948A7E0C94377E03E0068380
:10E6800008950CE417E490CD4D925D926D927C92CA
:10E6900013970895ECCD01E080160FEF90060895D2
:10E6A000FD011581011709F421DF0895FEDE80E5E3
:10E6B00093E023E030E00CE417E40E94D17DFC01FC
:10E6C000008B118BA089B18911971CF40FEF1FEFFC
:10E6D000F8CDAEE0B5E0FD0102A5002369F450D00D
:10E6E00059F5FD0103A514A5012B31F512A103A1D4
:10E6F0005BDD012B69F0C0DFFD0102A50230E1F412
:10E7000002E035D0C9F4FC0101851285012B19F016
:10E7100000E010E0DDCF26D0FD0103A5006403A7D3
:10E72000FC01408951899B969D010185C0DEFC0159
:10E7300026DE20D01C93ECCFFC0187DDFD01428D4D
:10E74000538D648D758D041715072607370729F03B
:10E750000F3F1F4F2F4F3F4FD9F600E0FC010487BA
:10E76000E5DED6CF08E412E0018712870895DADDEE
:10E7700000230895A185B285AA5FBE4F0D93089529
:10E7800000E0F5CF93DF012BF1F1A6DD0023D9F1F5
:10E7900090DE0AE010E0028B138B168B06810330AB
:10E7A00011F0043039F4048503950487023369F4C9
:10E7B00004E0068307811085012BC9F025D019F5E7
:10E7C00005850A3059F466DF11C0063999F740E132
:10E7D00030E007E411EE21D01CD05CCF00E00387CD
:10E7E0000585039505875BDD012B69F045CF068123
:10E7F000023011F0043039F407D029F400E0038727
:10E80000CBDC012B99F708950385039503870A3024
:10E81000089508EB1BE00C94287720E80C94107402
:10E820005B2F2A2E632F0EC0F80127FF008027FDE3
:10E83000049070E0A60FB71FFD0104820F5F1F4F09
:10E840002F4F6395342F4A95A7E6B3E0332361F742
:10E85000603238F400E0FD01E60FF01F0483639599
:10E86000F7CF01E0FD0107A308E813E12CD1A22DA9
:10E87000B52F089501D000D00C941F7818D01B98A4
:10E880001C9808B3036008BB36D002D00DD0F2CF7D
:10E890001D98F2CF8A93802F0AD01B980CC08A93C0
:10E8A000802F05D01B9A07C008B30F6008BB07B3C1
:10E8B0000F6007BB08951C9808B3007F08BB082FA2
:10E8C00002950F7018B3102B18BB0FD0007F08BB38
:10E8D0008F7008B3082B08BB08D00F6008BB07B3C4
:10E8E0000F6007BBD4DF89910895C6DF05D01D985E
:10E8F000C3DF08B30895C0DF1D9AC9CFE4E0F0EE8E
:10E9000088D0CDCF37D000A5002300E011F000A7BC
:10E9100001E00895E7E6F3E007A1002331F4008168
:10E920001181012B11F0EED011C000E007A31ED021
:10E9300002B1077C02B908B3007F08BB07B3007FB0
:10E9400007BB1A9A0AE03AD007EA14E70EC170D062
:10E9500061F01A9802B1086302B908D0A5DF0AD0A5
:10E9600004E12CD00DEB14E700D1089503B1077C2E
:10E9700003B90895E7E6F3E008955AD031F01D9801
:10E980001C9819D006EC14E7F0D0089551D039F056
:10E9900003D1F0DF0AE012D000ED14E7E6D00895CD
:10E9A00047D039F0FAD0E6DF0AE008D002EE14E7EB
:10E9B000DCD008952ED1E7E6F3E001E005A300E006
:10E9C00000A7089535D039F000E4F4DF0CEE14E729
:10E9D000CCD000E004A3089529D0D1F0A7E6B3E09D
:10E9E000FD0104A1102F139514A3E4E0F1EE11D062
:10E9F00056DF37D0FD01E2DF04A1069506950695A6
:10EA0000043018F00EE015E702C00CEE14E7ADD0AC
:10EA100057C010E0E00FF11F0491089509D029F0CC
:10EA200000E8C8DF0BE115E7A0D00895BA93AA93D8
:10EA300069DF00230895FADF99F05ED021F000E04D
:10EA400097960C93979701E094960C9390970C915E
:10EA500091965DD006D02FD0969704E315E733D07A
:10EA60002FC0A7D001E00895E1DF21F1A7E6B3E0D0
:10EA700094960C919497003228F497961C9197974E
:10EA8000112321F03FD012961ED014C0003131F472
:10EA900000EC8DD03DD006E615E7F6CF202F03958C
:10EAA00094960C93949710E0FD01E20F2ED0D9DFDD
:10EAB000959601D005C00C93139600E00C93089531
:10EAC000A991B99108950D931C930895AFDF99F022
:10EAD00013D019F017D012960DC094960C91102FE8
:10EAE00013951C93949710E0FD01E00F0ED010D009
:10EAF00004E315E7E8DFE4CFA7E6B3E097960C91CF
:10EB0000979797CF0AE814E70895F11F0481F6CE8E
:10EB100050D001E09596CFDF96970895E7E6F3E0B1
:10EB200000811181012B09F423D000811181015052
:10EB300010400083118305A1002311F401E040CFB0
:10EB40000A9505A3089502B10C6302B907B3007FCB
:10EB500007BB0CDFE7E6F3E000E007A304A308D05F
:10EB600000E006A305A300A7CDDF02831383089569
:10EB700008E813E10083118308958A93E4DF1A986B
:10EB800086E917D08A95E9F707D08DE212D08A95E9
:10EB9000E9F703D00ED0A7CE71CE0AD00AD008D0A4
:10EBA00000E237D008E235D00CE033D000E872CE76
:10EBB000F3DF0C9459780E94827ED801922F432E65
:10EBC000313210F000E01FC000E823D080E00FC019
:10EBD000803109F41DD050E0FD01392FE80FF51FF9
:10EBE000351F37FF008137FD049110D083958415C0
:10EBF00078F3803238F4803109F40AD000E206D08C
:10EC00008395F7CF01E0E5E00C948F7E80DFD1CFD4
:10EC100000ECCDDFCECF0E947B7E480159012A0156
:10EC20000FEF80169006A006B00671F400E02FEFFB
:10EC300010E0FA01E00FF11F208399D0C0F300E04B
:10EC400010E0ECE00C94887E80E993E093D009F426
:10EC500074C02AE933E000E011E0F9010687178764
:10EC600008E010E0008B118B06E0028B04E0038BC0
:10EC700000E011E0048B158BA4ECB3E050E0FD0143
:10EC8000E00FF51F6181F901E00FF51F668B6FD072
:10EC9000A8F367D0F901448F558F668F778F00E016
:10ECA0004FEFF90110E0E00FF11F40A360D0C0F377
:10ECB000F90186A297A2A0A6B1A66624C0D020E042
:10ECC00030E0C2D01123CAF148EE53E028E036E02C
:10ECD00000E013E80E94637AA801013010403CF183
:10ECE0000EE0002E05E0102EF00106A117A120A5D0
:10ECF00031A537D00417150726073707B1F4F001FF
:10ED0000348925892230304081F494D0FC0100837D
:10ED100011832283338300E030E0F0011FD0468965
:10ED20001CD0448324D048F4F7CF40E050E06394F3
:10ED3000452B19F40AE0601608F21CD019F00FEF09
:10ED40001FEF7FCF00E030E008D01481F20106D041
:10ED500010830DD008F073CFF6CFFC01E00FF31F46
:10ED60000895FD0147815085618572850895039559
:10ED700006300895FC01008111812281338108153C
:10ED800019052A053B0508950E94837E84EC93E0D3
:10ED9000FC010781108521853285AEE0B5E0FD01DB
:10EDA00046A157A160A571A54017510762077307D7
:10EDB000D1F55489458960E041305040A1F54AE9D8
:10EDC00053E071E0FA016687778768E070E0608B56
:10EDD000718B66E0628B64E0638B60E072E0648B51
:10EDE000758B1124FC0123D0218020D0268A6395C5
:10EDF0006630B8F3FA01048F158F268F378F60E0E5
:10EE0000FD0115D0268912D020A363956630C0F38A
:10EE1000FD0110D0FA0106A317A320A731A70FD038
:10EE200056969D0111D0E4E00C94907EFA01E60F15
:10EE3000F11D0895048D158D268D378D08956CE193
:10EE400070E048E056E0089500E013E80C94E279A1
:10EE5000E4ECF3E015C0E4ECF3E00689002300E005
:10EE600011F0068B01E00895E4ECF3E004EF11E00B
:10EE700007D0158B0895D1D0DED008EB1BE0FD0143
:10EE8000038B148B00E0068B08950D0100E0A4ECC9
:10EE9000B3E050E024E231EEF901E00FF51F3C96BB
:10EEA0001491FD01E00FF51F11830395063088F3DF
:10EEB0000FE00C93F90118D0478350876187728760
:10EEC000F901349611D04387548765877687F90115
:10EED00038960591159125913491FD010787108B86
:10EEE000218B328BD0010895459155916591749194
:10EEF000FD010895CADF43E150E024EC33E000E077
:10EF000010E00C94D978002309F4BFCF20E0022E42
:10EF1000112470E0622FAB010E945D7EF001EC5382
:10EF2000FC4F00832395233190F30091C4030F3FDE
:10EF300009F4E0CF0A3A19F00FE00093C4030895F2
:10EF40000E94817E2297A4ECB3E0FD01038914891D
:10EF5000012B19F401E0068B05C003890150104014
:10EF6000038B148B78DF002309F453C0FD0105895E
:10EF70000A9539F00A95E9F00A95A9F10A95F1F197
:10EF800048C080E593E0FC010681023050D059F082
:10EF900006E311EE20E84FD0FC01008111812281AF
:10EFA00033813BD003C007E411EE20E865DF02E0C7
:10EFB0002FC03DD000E011E03DD080E190E0FD01A8
:10EFC00010E0E90FF11F01810E941E7E0883198362
:10EFD00042E0382F8E012ED08E5F9395963078F3D5
:10EFE0004CDF03E015C023D001E111E026D00781FA
:10EFF0001085218532853FDF04E00AC018D002E287
:10F0000011E01BD0038514852585368534DF01E0AA
:10F01000058B2296E6E00C948E7E0E943B7B2801B5
:10F020000E94D37E402F30E1820120E0089540E12C
:10F0300030E0089520E00C941074FCDF59CF0000FC
:10F0400000000000000000000000000000000000C0
:10F050000895F5DFF4DFF3DFF2DFF1DFF0DFEFDF5C
:10F06000EEDFEDDFECDFEBDFEADFE9DFE8DFE7DF54
:10F07000E6DFE5DFE4DFE3DFE2DFE1DFE0DFDFDF84
:10F080000000000000000000000000000000000080
:10F0900000000895DEDFDDDFD2DFD1DFD0DF00004A
:10F0A0000000000000000000000000000000000060
:10F0B0000895CFDFCEDFCDDFCCDFC1DFC0DFBFDF24
:10F0C0000000000000000000000000000000000040
:10F0D00000000895E1E4F6E000811181012BE1F4E4
:10F0E000009156030330B1F00430A1F041E050E04C
:10F0F00020E030E004EC13E00E94FB78012B39F4AF
:10F100000091C4030A3A31F40C94000003C00FE0EC
:10F110000093C40349D003C0008101501040008314
:10F1200011830895BA93AA9300EC05BF04E00093FD
:10F130006D008F9A9798C79ABF980E941F7806B360
:10F140000078C798BF980E9483770E94BD753FE101
:10F1500008E511EE20E80E94DB7500E013E80E944C
:10F160008279012B49F00E94BD7539E003E311E07B
:10F1700020E00E94DB75FFCF0E944C710E94347723
:10F1800013D0008311830E94C2730E948E7CA9E673
:10F19000B3E0ED91FC9109950E94A0770E948E75D5
:10F1A0000E94747197DFEFCF08E813E1E1E4F6E025
:10F1B00008950E94837ECA01D801F9019801183090
:10F1C00010F431D078F40FEF1FEF12C09D010081D1
:10F1D000A9010E94697EA9010E945D7E119101171B
:10F1E00091F711968C010197012B81F700E010E057
:10F1F000E4E00C94907E0E94837ECA01F801D9015C
:10F20000383010F410D040F40FEF1FEF0BC0AD01F9
:10F210000E945D7E019311968C010197012BB9F735
:10F2200000E010E0E5CF00E018E0021B130B04172C
:10F230001507089548E05C9156275D934A95D9F7E4
:10F240000895772359F02D903C9030FA2794379405
:10F2500027F87A95D1F73C922E9211960895AA93A9
:10F26000BA938A93F9011590712D72957F70B1F060
:10F27000072E6AEAD801712D7F70E3DF83E0749175
:10F2800072957F70DEDF75917F70DBDF8A95B9F74D
:10F29000D801D0DFF90115900A9461F78991B991ED
:10F2A000A99108958DD0D80180E0979A04E610E0E6
:10F2B0001FD0979821D0978D1FD0978F90E004ECA6
:10F2C00019E01CD0078107FF08C00285003529F42A
:10F2D0000385003711F4F1D008C09395943178F389
:10F2E0008395843110F30FEF1FEFE4E00C94907ED0
:10F2F00020E030E00C94007E04EF11E020E0F9DF24
:10F30000FD0108955DD0D801CDDF012B19F00FEF7D
:10F310001FEF55C000E0FD0107870FEF078301EEE7
:10F320000C9300EC018300E0068300E2058300E01B
:10F33000018304ED10E3DCDF01E20C9308E4FD013E
:10F34000068700E00287038700E2048702E0058762
:10F3500000E404830FE503830CE4018300E60283E9
:10F360000FEF078301E60C93ABD0FC01EC53FC4F8D
:10F370000181FD01E80FF91F01830196863000E04D
:10F38000900798F39DD0FD01E80FF91F00870196C3
:10F3900088309007C0F30CE4FD01078301E20C9371
:10F3A00004E004870FEF078300E0078702E20C9375
:10F3B00000E0058700E211EA27E09BDF7ED095CFD1
:10F3C0000C94837EFDDF09011A01483026E03206E5
:10F3D00019F42AE933E002C02BED33E0F90170D0D3
:10F3E000DC01AB53BC4F5C91D9011696A80FB91F35
:10F3F0005C935ED0A8F3402D412962D039F0D00152
:10F40000A80FB91F4C9150D020F4F9CF4FEF4CD03A
:10F41000E8F3D9011C962D923C92625F7F4F6C33CA
:10F4200020E0720718F42CE330E001C09B0142E2B7
:10F43000D8014C931A962C93D8011B963C9350E01C
:10F44000D80118965C9350E4D80119965C9352E168
:10F45000D8015C9335D005C05191D80150965C938A
:10F46000019686179707C0F3CB0104C050E0F8015E
:10F47000508B019682179307C8F3F801408320D080
:10F48000578156FD05C00196853150E09507C0F3C0
:10F4900050E4578325833683548326E220832081DA
:10F4A00022FDFDCF0AD021CFD901A80FB91F4C935F
:10F4B0000196863040E09407089500E010E008953A
:10F4C00080E090E008950E94817E2497D801290170
:10F4D000CA01F3DF01C04783282F292B09F454C048
:10F4E000202F212B09F050C021E008C0222309F46D
:10F4F00001972395382F392B09F445C0FD01478129
:10F5000042FB16F434E0378340FB86F722E62C9367
:10F51000578122E22C9333813395303608F03CE456
:10F520003517C9F224E0228720E02387208731871E
:10F53000BE012AE02C9324E0FD015089FB01519388
:10F54000BF012A95C9F722E22C9300241124FD0162
:10F55000278126FD09C021E0020E20E0121E25E1D0
:10F56000021620E0120698F320E427830A801B800D
:10F57000021620E0120628F023EF021625E01206FC
:10F5800038F09BDF01C047832496E6E00C948E7E22
:10F59000002011F051E001C050E0212D230F250F74
:10F5A000203608F024516981261741F02395522F07
:10F5B000203608F05451561731F7252F4EE055E00C
:10F5C00068816F70613099F58001045010400287A6
:10F5D000138764E0608731873AE03C93BA010024E6
:10F5E000112401C036D00016110658F433E3031677
:10F5F00031E01306FD013089A8F7FB013193BF010B
:10F60000F1CF043331E0130710F003E311E032E2ED
:10F610003C9300241124FD01378136FD06C019D02A
:10F6200035E1031630E01306B0F330E437832A9552
:10F630002C3408F42FE52383FA012485358524151D
:10F64000350509F449CF2830364011F40E94C476BC
:10F6500040CF31E0030E30E0131E0895F80103C0DF
:10F66000F801090121E020936800E89520916800E5
:10F6700020FDFCCF08950E947F7E27970B831C837B
:10F680002D833E83A3E4B6E02E0103E0400E00E0AC
:10F69000501E94E080E0F201608026D0742E24D0C9
:10F6A000F201008310E3710EFE0130E0E80FF31F5A
:10F6B00070828395002379F7082F8A95002331F013
:10F6C000FE01E80FF31F00810D93F6CF0EE20D93BC
:10F6D00001E0400E531E9A95E9F63E9303E416E0CE
:10F6E0002796E8E00C948C7E062D4AE00C946D7E03
:10F6F0000801890140E050E060E070E0F00108C0DE
:10F7000001901190400D511D621F721F0250104058
:10F71000023020E01207A0F7012B51F00081400FCA
:10F72000521F621F721F04C0460F571F60E070E037
:10F73000262F272BC9F70FEF1FEF04271527089552
:10F740000E94847EA02FC901AC0128E030E000E0D7
:10F7500013E80E94637A312F01303040F4F1EEE07B
:10F76000F5E02685022F007F003471F714890589A2
:10F770001F73012B49F707890A1731F7108901898F
:10F780002F7034E0239F00191040068C178C20A0A6
:10F7900031A02FEF0216120622063206F1F0E4EC39
:10F7A000F3E04781508561857285242F252B262B18
:10F7B000272B51F2041615062606370671F04385ED
:10F7C00054856585768540295129622973294F3FE3
:10F7D0005F4F6F4F7F4F09F0B7CFE3E00C94917EFE
:10F7E0000E947E7E269728013901842ECB01AE012E
:10F7F0000E940B76012B19F00FEF1FEF34C0ABED19
:10F80000B3E005E4FD0106874496908B818B00E40C
:10F81000068B878A468E578E60A271A2E4ECF3E0D5
:10F820000781108521853285FD01028F138F248F7A
:10F83000358F028913890F5F1F4F028B138B00E0F6
:10F84000008F018F24E130E08D01025F1F4F50DFF8
:10F85000FD01008F118FBC0148E050E09E0100E0E7
:10F8600013E80E94E2792696E9E00C948B7E9A9345
:10F870008A9380E090E028E731EE05E516E0080F76
:10F88000191F0D5F1F4F0E942F790896913098F332
:10F890008991999108950E947F7EA02FCA01290124
:10F8A000413001E0900710F080E091E0BA2FA0E035
:10F8B00023E01ED06624772405C0F2012191319106
:10F8C0002F010FD068167906C0F301E0701620F4FE
:10F8D0002FEF3FEF06D0F9CF25E00AD0E8E00C94F7
:10F8E0008C7E83010E94307B02E0600E7A1E0895B8
:10F8F0008D010E942E7B21E100E010E00C942E7B14
:10F90000E3E5F6E000810E7F026000830FEF0383E2
:10F91000048325E030E08F010C94E1710E94817E28
:10F92000239783E596E026E031E08C010E9429725E
:10F93000280101E0401600E0500634F40FEF1FEFFD
:10F940002396E6E00C948E7E10D107FFF7CFE0E51A
:10F95000F3E007811085012B89F7FC010181002369
:10F9600021F00F3F11F0CCDFE9CFABE5B7E002812A
:10F97000005F09F488C00A9509F4A4C00A9509F447
:10F98000DEC00A9509F47FC00B50C1F00A95E1F181
:10F990000A9541F00A9549F00F50E1F10A9509F4F2
:10F9A00055C0DCC000E010E0CBCF008100FFFACFF3
:10F9B000E9D092018C010E94E171F4CF008100FF37
:10F9C000F1CFE0D002E0400E00E0501E41E050E0F8
:10F9D00020E030E004EC13E00E94FB78012B39F0CA
:10F9E000C7D0008302E0038302E80483E2CF0091E2
:10F9F000C4030A3A19F40C940000D4CFB9D00083A0
:10FA000001E0038303E8F1CF008100FFCBCF0E9428
:10FA1000377EC8CF008100FFC5CFB4D04581568165
:10FA20009C01295F3F4F148103810E94D9789CD0AB
:10FA300049F0ABD001E0FC01038302E8048329E034
:10FA400030E0B8CF0D7F008327E0FACF008100FFC0
:10FA5000A9CF98D0A581B681B13018F096D003E037
:10FA6000EACFAD01348123818C01095F1F4F0E94D1
:10FA7000FB787AD019F089D002E0DDCF0D7F0083CA
:10FA800017969D0197CF008100FF8CCF7BD003811B
:10FA9000013011F0002371F4FD01028300E00D93A9
:10FAA0000C93FC01048301E0058300810D7F00833A
:10FAB00026E0C6CF01E0038301E8048301E005836B
:10FAC00058D0F5CF008100FF6DCF5CD049D0012B1D
:10FAD00099F40FE00093C40341E050E024EC33E0DC
:10FAE0004BD051F042E050E054D003E0FC010383DE
:10FAF00001E804833ED0A7CF33D0003E50E0104051
:10FB0000D0F4FD010281002309F0B1DE0BEF400EBD
:10FB10000FEF501EA2019C012B5F3F4F21D0BBDE97
:10FB20000D911C910F5F1F4F1C930E931ED00D7FE4
:10FB3000008325E085CF42E02CD002E0D7CF0081C2
:10FB400000FF30CF1FD00AEA088341E050E09E0159
:10FB500013D061F30FE00093C403C4CFD1DE22CFF2
:10FB60000D911C9111970895012BFC0100810895BE
:10FB7000FC0100810260089500E010E00E94D97845
:10FB8000012B08950E7F008308950260008344E0F6
:10FB900050E09C012D5F3F4F8C010B5F1F4F0C9479
:10FBA0009D7E0E94817E2801C9019C0101E10E9485
:10FBB000A07BD8010130104054F0EEE0F5E034A114
:10FBC00005A14016530689F7B6A1A7A118978D0184
:10FBD000E6E00C948E7E9A938A938A819B81EBED6A
:10FBE000F3E072A363A354A345A3089696A387A347
:10FBF000BC0141E10E94F07B899199912296089580
:10FC0000249740E0488349834A834B830AC000001D
:10FC100010D04F5F5F4F6F4F7F4F488359836A8388
:10FC20007B8307D0401751076207730784F324963C
:10FC30000895488159816A817B8108950E94837E5D
:10FC4000E02FE295EF70AE2FB0E0EA3010F4D096DE
:10FC500001C0D796802F8F700F700A3010F4805D2E
:10FC600001C0895CB82B8D01E4E00C94907E01B555
:10FC7000086101BD01B5086101BDFFCF0000889595
:10FC8000FECF0DE90DBF07E00EBFCEE9D9E00E941F
:10FC90009B7E002311F00E94B97E0E9492780E9400
:10FCA0003E7E0C943E7EE199FECF08954F5F5F4FFC
:10FCB000FADF4EBB5FBBE09A0895FADF0DB30895FB
:10FCC0004F5F5F4F4EBB5FBBF894E29AE19A0FBE65
:10FCD00008950FB6E8DF0DBBF5CF0024E8E0EA9504
:10FCE00032F0001F001C0416D0F3041AF8CF001FD6
:10FCF000402D00950895BA92AA929A928A927A9289
:10FD00006A925A924A92BA93AA939A938A930895BE
:10FD1000BB84AA84998488847F806E805D804C80B7
:10FD2000BB81AA8199818881F0E00FB6F894CE0F4B
:10FD3000DF1F0FBE089501E008950D01D80104C032
:10FD4000F90161919F016D93BA0141505040672BB9
:10FD5000B9F7D001089520E006D0E9F7089525917C
:10FD600002D0E9F708952D9301501040202F212B48
:10FD700008958CE891EEFC0105911491FC013296F6
:10FD8000A591B491FC01349625913491422F432BD7
:10FD900019F0F901E4DF01C0DEDF069611EE8839C3
:10FDA000910748F30895F80101C03196208122237C
:10FDB000E1F7E01BF10B8F0108954574686572420D
:10FDC0004C204D41433A2020202000457468657244
:10FDD000424C2049503A202020202000457468657C
:10FDE00072424C204950204D41534B3A004E4943FA
:07FDF000204552524F520062
:00E000011F
:00000001FF
